:104F9A000000090101240200000301FA0400FA05D5
:104FAA0000020A0A5A0B000F0C00FA0D00030E0049
:104FBA00030F0132100096120132130AFA14010289
:104FCA0015000217010A18010A1905321A010A1BEB
:104FDA00010A1C053223011E2400642A00FA2B0050
:104FEA00FA2C50782D003C2E00462F001E3000640B
:104FFA003250783300003432FA35016436016437AE
:10500A000150380A643C00643E003C3F000140FF06
:10501A00FF411450420A5A430AC8440532450078EF
:10502A004600FA4701234802034C00FA4EFFFF509C
:10503A000808510596520A32530B28540A9656010B
:10504A0002570546580002590A465A32FA5B010AC3
:10505A005C0A325E000A5F00FE61FFFF64021166AD
:10506A0000016701036A0A3C6B00006C3296780102
:10507A0032790132FAFAFA00000901012402000029
:10508A000301FA0400FA0500020A0A5A0B000F0C7F
:10509A0000FA0D00030E00030F01321000961201F0
:1050AA0032130AFA14010215000017010A18010A3C
:1050BA001905321A010A1B010A1C053223011E2492
:1050CA0000642A00FA2B00FA2C50782D003C2E009E
:1050DA00462F001E3000643250783300003432FA12
:1050EA00350164360164370150380A643C00643E75
:1050FA00003C3F000140FFFF411450420A5A430A54
:10510A00C84405324500784600FA4701234802029E
:10511A004C00FA4EFFFF500808510596520A3253C6
:10512A000B28540A96560101570546580001590A98
:10513A00465A32FA5B010A5C0A325E000A5F00FED6
:10514A0061FFFF6402116600016701036A0A3C6B92
:10515A0000006C3296780132790132FAFAFA006567
:10516A00006F00790083008D009700A100AC00B6A3
:10517A0000C000CA00D400DE00E800F2005B006351
:10518A00006A0072007A008200890091009900A1E9
:10519A0000A800B000B800BF00C700CF00D600DFEB
:1051AA0000E600EE00F600400046004C00520059AE
:1051BA00005F0065006B00710077007D0083008945
:1051CA00008F0095009C00A200A800AE00B400BAAF
:1051DA0000C000C600CC00D200D900DF00E500EB19
:0251EA0000F1D2
:10009E0085F95085FA517E017F00E551125476E5BF
:1000AE00502FFF50010E8E338F3490001CE0FCA3B6
:1000BE00E0FDEF2DFDEE3CFC8C358D362275A71044
:1000CE0085F95085FA517E017F00E551125476E58F
:1000DE00502FFF50010E8E338F3490001CE0FCA386
:1000EE00E0FDEF2DFDEE3CFC8C358D3622AE33AFB0
:1000FE0034740A8E048F05FF1254588C358D36AE2B
:10010E0033AF34740A8E048F05FF1254918C338DE5
:10011E0034E53445336013740AC39534FFE49533E4
:10012E00FE8E338F3478351254D3E550A835B8008F
:10013E0015D395364010E550C39536FFE49535FE40
:10014E008E358F368010E5502424C39536FFE49506
:10015E0035FE8E358F36AE35AF3674246F4E700B3E
:10016E007536237535007550018003755000229049
:10017E00008FE0B40104C20B8002D20B900090E01D
:10018E00B40104C20C8002D20C9000CDE075F0DCFC
:10019E00A4FFAEF0740A8E048F05FF125458900718
:1001AE00B5ECF0A3EDF0A208401674038C068D0793
:1001BE0012547674011254689007B3EEF0A3EFF068
:1001CE007E017F0090008BE01254769000CEE08E80
:1001DE00048F05FF125458740AFF1254588D39902B
:1001EE0000D7E075F0DCA4FFAEF0740A8E048F0524
:1001FE00FF1254589007B9ECF0A3EDF09000D9E03F
:10020E0060139000D9E0F5F0741684FF7E00EF9035
:10021E0007C1F0800674649007C1F09000E1E0B46D
:10022E00010674009000B5F09000B8E0B40B0874AD
:10023E00E390007AF080499000B8E0B41912900073
:10024E00CEE090515312008CE49390007AF08030FF
:10025E009000B8E0B41E129000CEE09051711200E2
:10026E008CE49390007AF080179000B8E0B42810D8
:10027E009000CEE090519B12008CE49390007AF0A7
:10028E00900056E0C39405502274019000D1F09076
:10029E0000D3E0B4020674019000D3F09000C3E0E6
:1002AE00D39402400674029000C3F09000EBE0B4C9
:1002BE000117900028740FF0A374FFF090002AE449
:1002CE00F0A3F074029000EBF09000EBE0B4034169
:1002DE0090002AE0FEA3E0FF900028E0FCA3E0FDE2
:1002EE001254CB74101254767408125468EF9000A6
:1002FE0077F0EF700674FF900077F074009000EBCB
:10030E00F0900029E0900078F0900028E0900079BD
:10031E00F090007CE090003CF090003CE0240990CE
:10032E00003DF090003CE0241290003EF090003C26
:10033E00E0241B90003FF090003DE0D39424400B4E
:10034E0090003DE0C3942490003DF090003EE0D339
:10035E009424400B90003EE0C3942490003EF09015
:10036E00003FE0D39424400B90003FE0C3942490D0
:10037E00003FF0900044E4F090003CE0B4240C9078
:10038E0000447401F090003C7401F0900045E4F0DC
:10039E0090003DE0B4240C9000457401F090003DB7
:1003AE007401F0900046E4F090003EE0B4240C900E
:1003BE0000467401F090003E7401F0900047E4F0A6
:1003CE0090003FE0B4240C9000477401F090003F81
:1003DE007401F090007CE0FE9000DFE02E9000496A
:1003EE00F0900049E0D39424400B900049E0C39470
:1003FE0024900049F0900049E0B412067413900066
:10040E0049F0900049E0B424069000497401F09040
:10041E000049E0D39412400D900049E0C39412902D
:10042E00004AF0800A900049E0241290004AF090B1
:10043E0000C2E0900040F0900040E06409600F9030
:10044E000040E064126007900040E0B41B0690008C
:10045E0040E004F0900040E02409900041F090004C
:10046E0040E02412900042F0900040E0241B9000E7
:10047E0043F0900041E0D39424400B900041E0C340
:10048E009424900041F0900042E0D39424400B90CD
:10049E000042E0C39424900042F0900043E0D394D5
:1004AE0024400B900043E0C39424900043F022C2FA
:1004BE0093C294C291C292C287C290E5B554EFF531
:1004CE00B5E5B554DFF5B5C296C295C2A0C297C2C6
:1004DE00A2C2A1E5B554BFF5B5E5B5547FF5B5E5B6
:1004EE00B554FBF5B5C20D7537469000C5E07005E5
:1004FE00754902800375490390001074FFF0A374D0
:10050E00DCF09000A6E0900016F8E4F0E8A3F0C24C
:10051E0014C216C218C21A74C890002CF074C89077
:10052E000030F074C8900034F074C8900038F07544
:10053E002600752500C208756C00E54BB4090375DD
:10054E004B00753C0090001EE4F0A3F0754C1E7538
:10055E002800752700C210C211C212C2139007B52F
:10056E00E0FEA3E0FF7403125476740112546890F7
:10057E0007B3EEF0A3EFF0C203900014E4F0A3F083
:10058E00C2252285F95085FA517E017F00E5511270
:10059E005476E5502FFF50010E8E338F349007B5F1
:1005AE00E0FCA3E0FDEF2DFDEE3CFC8C358D36E539
:1005BE0036F5FDE535F5FE22053D229000C3E064DB
:1005CE000360079000E1E0B4021EA2D8B34002C25D
:1005DE0093A2D9B34002C294A2DAB34002C291A24E
:1005EE00DBB34002C292802CA2D8B34004C293C2A5
:1005FE0087A2D9B34004C294C290A2DAB34008C213
:10060E0091E5B554EFF5B5A2DBB34008C292E5B55E
:10061E0054DFF5B5A2DCB34008C296C295C2A0C2A3
:10062E009775D8402285A74F75A7109000C3E0B4E8
:10063E000324A2D8B34002C287A2D9B34002C2900B
:10064E00A2DAB34006E5B554EFF5B5A2DBB340062A
:10065E00E5B554DFF5B575D840854FA72290004714
:10066E00E4936406600280FE74C89007BBF8E4F061
:10067E00E8A3F075B50075840175A70075FF807548
:10068E00EF06900048E4F075C91075A70F75A1C765
:10069E0075A70075D90075CE0C75A70F75F1FE758F
:1006AE00F2FF75F30775F47875A4BA75A5FF75A6F4
:1006BE000775AE0075AFFF75D48175D5FF75D6FF82
:1006CE0075D7FF75A70075A20175A14775F8097555
:1006DE00D80075D90475DA0975DB0975DC0975DD85
:1006EE000975DE0975D84075A71075D80075D9043F
:1006FE0075DA0975DB0975DC0975DD0975D8407584
:10070E00A70075E60875E71075BC0175BE0475BDCA
:10071E006C75BE0775BDA075BE0875BD0175BC00B4
:10072E0075BB1875BC2075BA0875E88075D1137540
:10073E00A70F75E10575E20075C740C293C294C25A
:10074E0091C292C287C290E5B554EFF5B5E5B554A6
:10075E00DFF5B5C296C295C2A0C297C2A2C2A1E5EC
:10076E00B554BFF5B5E5B5547FF5B5E5B554FBF514
:10077E00B5759700759780740A1254487597C0E541
:10078E00975420700280F8758F0275A700D2AF754E
:10079E00980075A90C75A70F75AB4375ADFB75ACBD
:1007AE001E75A71075C91875CA0075CB0075C804DB
:1007BE0075A700758912758E04758C00758A00C236
:1007CE00A9D28C758D00758B00D2ABD28E75D944A3
:1007DE00753200753100752E00752D007546007549
:1007EE004700C29974C8F5097508001233A675B58D
:1007FE000074639007BBF8E4F0E8A3F0123632748D
:10080E0064F5097508001233A6C21F900065E0B4A6
:10081E000108A2B54002D21F802E900065E0B402FE
:10082E001175A70F75F30F75A700A2A34002D21F73
:10083E008016900065E0B4030F75A70F75F317755A
:10084E00A700A2A44002D21FA21FB3500302094464
:10085E0074089007BBF8E4F0E8A3F0123501746455
:10086E00F5097508001233A674099007BBF8E4F079
:10087E00E8A3F01235017464F5097508001233A669
:10088E00740A9007BBF8E4F0E8A3F0123501746423
:10089E00F5097508001233A6740B9007BBF8E4F047
:1008AE00E8A3F01235017464F5097508001233A639
:1008BE00740C9007BBF8E4F0E8A3F01235017464F1
:1008CE00F5097508001233A6740D9007BBF8E4F015
:1008DE00E8A3F01235017464F5097508001233A609
:1008EE00740E9007BBF8E4F0E8A3F01235017464BF
:1008FE00F5097508001233A674029000C4F090003A
:10090E0065E0900088F0900065E0B40108740090F6
:10091E000090F0801C900065E0B402087400900016
:10092E00D3F0800D900065E0B4030674009000E0F3
:10093E00F0D21D020A249007BBE4F0A304F0123596
:10094E00017464F5097508001233A674029007BB92
:10095E00F8E4F0E8A3F01235017464F509750800A7
:10096E001233A674039007BBF8E4F0E8A3F0123537
:10097E00017464F5097508001233A674049007BB60
:10098E00F8E4F0E8A3F01235017464F50975080077
:10099E001233A674059007BBF8E4F0E8A3F0123505
:1009AE00017464F5097508001233A674069007BB2E
:1009BE00F8E4F0E8A3F01235017464F50975080047
:1009CE001233A674079007BBF8E4F0E8A3F01235D3
:1009DE00017464F5097508001233A674019000C401
:1009EE00F0900065E0900088F0900065E0B401089A
:1009FE007400900090F0801C900065E0B4020874C2
:100A0E00009000D3F0800D900065E0B403067400F2
:100A1E009000E0F0C21D1237A69000CEE070067472
:100A2E000A9000CEF090007AE0700674E390007A9F
:100A3E00F012017DE5B54401F5B57406900054F051
:100A4E007401900055F07403900057F074049000F8
:100A5E0058F07410900059F0740590005AF0900000
:100A6E0056E0B40406740490005AF0740690005BCD
:100A7E00F07400900060F07400900061F0740190CA
:100A8E000062F07400900063F074FF900064F074E4
:100A9E0033900152F07436900153F0742D9001543E
:100AAE00F07431900155F07420900156F074389026
:100ABE000157F07443900158F07479900159F07415
:100ACE006C90015AF0742090015BF0742090015CE0
:100ADE00F0742090015DF0742090015EF07420900F
:100AEE00015FF07420900160F09000EAE0900077D2
:100AFE00F09000A1E0900078F09000A2E0900079D4
:100B0E00F0C214C216C218C21A74C890002CF07427
:100B1E00C8900030F074C8900034F074C89000385B
:100B2E00F0C210C211C212C213A2B6B39209A2B37E
:100B3E00B3920A752600752500753746754C1E90C2
:100B4E000073E4F075271975286490001074FFF097
:100B5E00A374DCF0C20D754B00C208752A0075290E
:100B6E0000900014E4F0A3F0743A90077BF074FD4B
:100B7E0090077CF0756D00900074E4F0752C007594
:100B8E002B00900018E4F0A3F09000A6E090001661
:100B9E00F8E4F0E8A3F0900087E075F032A4FFAE21
:100BAE00F0900026EEF0A3EFF09007B5E0FEA3E084
:100BBE00FF740312547674011254689007B3EEF06A
:100BCE00A3EFF0754A01900050E4F0C225C22275E1
:100BDE006C00753C00C20EC20FC226C203754D00DA
:100BEE00C204D205C206D207C220C221D21E74FE92
:100BFE0090004BF074FE90004CF0C223D224753856
:100C0E0000754400753A00753E32753F0075400020
:100C1E00743C90004EF0754100743C90004FF0759E
:100C2E00420075430090001EE4F0A3F0754500D21B
:100C3E00B2D2A4D2B0D2B1D2A3D2A7D2A6D2A5D2CA
:100C4E00B7900087E0D394FA400674FA900087F0CC
:100C5E007E017F00900079E0125476900078E02FAC
:100C6E00FF50010E900028EEF0A3EFF0EFD394FFAB
:100C7E00EE940F4007900028E4F0A3F0900077E088
:100C8E00700674FF900077F09000C4E0D394024099
:100C9E000674019000C4F09000C5E070057549021D
:100CAE0080037549039000C6E0D39401400674009A
:100CBE009000C6F09000CCE0C3940A5006740A90DF
:100CCE0000CCF09000D6E0700674019000D6F09043
:100CDE0000D6E0B4FF0674FE9000D6F09000DDE082
:100CEE00D394FE400674FE9000DDF074019000E394
:100CFE00F074019000E4F074009000E6F07400903F
:100D0E0000EBF0D29CD2EC75CF01A298B350030247
:100D1E00111AC298E54764046006E59964FF600203
:100D2E00802AA2234004D2238020E547600874E67F
:100D3E002547900050F0754700E546600874F02591
:100D4E0046900050F0754600C2238002C223E5474C
:100D5E006003020DFE754700E599B4FF0375460169
:100D6E00E599B4FE03754602E599B4FD0375460395
:100D7E00E599B4FC03754604E599B4FA0375460586
:100D8E00E599B4FB03754701E599B4F9037547047A
:100D9E00E599D394E54007E599C394F04002801697
:100DAE008599487547027E017F00E548C394E61297
:100DBE0054768E2F8F30753200753100E599D394AD
:100DCE00C74007E599C394E64002801F8599487590
:100DDE00470374E5C39548F530752F00AE2FAF303D
:100DEE009051EC12543778311254B1D29902111A33
:100DFE00E547B401028003020ED6AE31AF32900049
:100E0E007B12549DE599F078311254D3AE31AF3246
:100E1E00EFB40106EEB407028003020ED690077BF4
:100E2E00E0B43C028003020EC0C29C1204BD12014B
:100E3E007D900077E09000EAF0900078E09000A1BD
:100E4E00F0900079E09000A2F0A21D4032755001A2
:100E5E00E550D394075026E5509007BBF8E4F0E830
:100E6E00A3F074AA900048F01233D27464F5097599
:100E7E0008001233A67850740126F650D3803075D0
:100E8E005008E550D3940E5026E5509007BBF8E479
:100E9E00F0E8A3F074AA900048F01233D27464F50F
:100EAE00097508001233A67850740126F650D31235
:100EBE0037A674C89007BBF8E4F0E8A3F0D29C758F
:100ECE0047007546007599FBE547B40202800302A0
:100EDE000F77E5324531700685992E752D00AE31AE
:100EEE00AF3274016F4E701BAC2DAD2EAA2FAB30EE
:100EFE00ED2BFBEC3AFA8A068B0790007B12549D81
:100F0E00E599F078311254D3AE31AF3274026F4E90
:100F1E007057AC2DAD2E740D6D4C702C7463900704
:100F2E00BBF8E4F0E8A3F074AB900048F0900088B2
:100F3E00E0900065F012370B900048E4F074C89012
:100F4E0007BBF8E4F0E8A3F0AE2DAF2E74566F4E4B
:100F5E007006E54864E6600280031204BD12017D4E
:100F6E00854899754700754600E547B4033FAE3195
:100F7E00AF3290007B12549DE599F078311254D324
:100F8E00AE31AF32AC2FAD308F028E038C068D0793
:100F9E00905228125437E493F9740193FEEAD39ECB
:100FAE00EB994009854899754700754600E547B4A9
:100FBE000402800302111AAE31AF3290007B12543C
:100FCE009DE599F078311254D3AE31AF32EFB400C3
:100FDE0006EEB40102800302111A1204BD90005EE7
:100FEE00E075F002A4FFAEF08F50EF90007B12542C
:100FFE00A8EFFCE0FDEC90007E1254A8EDFCE0FDA5
:10100E00EC2DFC90005EE0B50402800302110B0F84
:10101E00EF90007B1254A8E550FFE0FCEF90007FAC
:10102E001254A8ECFFE0FCEFC39CFF90005EE0B50D
:10103E000702800302110BE55090007D1254A8E5C3
:10104E0050FFE0FCEF9000801254A8ECFFE0FCEFA4
:10105E002CFF90005EE0B50702800302110BE550F5
:10106E009000811254A8FFE0FCEF90005EE0F404C3
:10107E002C900065F0E5509000821254A8FFE0FC21
:10108E00EF90005EE0F4042C900066F0E5509000C6
:10109E00831254A8FFE0FCEF90005EE0F4042C9065
:1010AE000067F0E5509000841254A8FFE0FCEF902A
:1010BE00005EE0F4042C9007BBF8E4F0E8A3F074B3
:1010CE00AB900048F012370B7464F50975080012E6
:1010DE0033A69007BB12548412370B7464F509754E
:1010EE0008001233A69007BB12548412370B759961
:1010FE00F97464F5097508001233A680FE7599FF20
:10110E007464F5097508001233A680FEE546600684
:10111E00A299B3B3400302129AC299E546B4011FD5
:10112E00AE31AF3290005412549DE0F599783112E1
:10113E0054D3AE31AF3274116F4E7003754600E565
:10114E0046B40203854A99E546B4031DAE31AF326B
:10115E0090007B12549DE0F599EFB40107EEB407B1
:10116E000375460078311254D3E546B40402800369
:10117E0002125CE53245317003852699AE31AF32ED
:10118E0074016F4E7003853899AE31AF3274026FB1
:10119E004E7003853A99AE31AF3274036F4E7003C1
:1011AE00853E99AE31AF3274046F4E70038540990F
:1011BE00AE31AF3274056F4E7003854199AE31AFCB
:1011CE003274066F4E7003854299AE31AF3274079A
:1011DE006F4E7003854399AE31AF3274086F4E7007
:1011EE000690001FE0F599AE31AF3274096F4E7064
:1011FE0017A224B340077599FAC224800B900050B1
:10120E00E0F599900050E4F0AE31AF32740A6F4EB3
:10121E007003854499AE31AF32740B6F4E700385F7
:10122E003F99AE31AF32740C6F4E7003854599AE57
:10123E0031AF32740D6F4E70037599FC78311254C4
:10124E00D3AE31AF32740E6F4E7003754600E54665
:10125E00B40539900056E0D394044010AE31AF324D
:10126E00904F9A12549DE493F599800EAE31AF32A1
:10127E0090508112549DE493F599AE31AF3274E6DD
:10128E006F4E700375460078311254D3E5476401F2
:10129E006005E547B40403020D15C28E7E107F0073
:1012AE00E53D125476E58D75F010A4FDACF0EF2DF2
:1012BE00FDEE3CFCE58B75F01084FF7E00ED2FFFFC
:1012CE00EC3EFE8E278F28D28E9000A8E0605690BE
:1012DE000020125484900020E0FCA3E0FD90002238
:1012EE00E0FAA3E0FBEDB5033CECB50238B21CA26C
:1012FE0008B34013A21CB34008E5B54404F5B5800D
:10130E0006E5B554FBF5B5900022E0FEA3E0FF9094
:10131E000024E0FCA3E0FDEF2DFDEE3CFC9000224E
:10132E00ECF0A3EDF09000E1E060030213EA900010
:10133E00B5E060099000B5E0C394034002807A12D4
:10134E004CE0A208B35009900073E0C394464002EB
:10135E00800690009FE0F56BE56B75F005A4FFAE7F
:10136E00F09007BDEEF0A3EFF090008CE0C3953A3D
:10137E004007E538C3953950079007BDE4F0A3F058
:10138E00AE58AF599007BDE0FCA3E0FDEFD39DEE44
:10139E009C4004C2A1800B900073E0C39464500281
:1013AE00D2A19000B5E0B402099000D3E0C394023C
:1013BE0040028005A2A1B392A29000B5E0B4031C36
:1013CE00124DFBAE58AF599007BDE0FCA3E0FDEF08
:1013DE00D39DEE9C4004D2A18002C2A1900090E069
:1013EE006009A2B3300A01B3B340028039A2B33010
:1013FE000A01B34031A2B3300C01B3401C9000C3BC
:10140E00E0B40306A220B3B3400280067405900038
:10141E0050F0D220A20CB3920AA20CB330B301B397
:10142E004004A20C920AA2B6300901B35003021A6C
:10143E0036A2B6300901B35003021A36A2B6300BEB
:10144E0001B3500302194D754A009000A8E07013C5
:10145E00A20BB34008E5B554FBF5B58006E5B544DF
:10146E0004F5B50537A20DB3B35013AE27AF2890D0
:10147E000010E0FCA3E0FDEDC39FEC9E40030215BF
:10148E008CE549B40330E537B42405754901801F56
:10149E00A225B3401AE537C3942450069000507429
:1014AE0001F0E537D3942440067402900050F07595
:1014BE003701D225805EE549B402067549017537BC
:1014CE0024E537B424057537018049900050E0704B
:1014DE0034E537C3942450069000507401F0E5377C
:1014EE00D3942440067402900050F0E537C3942440
:1014FE005002D222E537D394244002D222C296C2A1
:10150E0095C2A0C2979000C5E0B402051204BD803A
:10151E0003753701AE29AF2AAC27AD28EF2DFDEEAE
:10152E003CFC7403FF1254588C298D2A9000A8E0BD
:10153E006043900020E0FEA3E0FF9000A8E08E0440
:10154E008F05FF12545874018C068D071254689043
:10155E000024EEF0A3EFF0900024E0F8A3E090005A
:10156E0022C8F0A3C8F0900020E4F0A3F0C21CE55E
:10157E00B554FBF5B5A222B34002C222802BAE2990
:10158E00AF2AAC27AD28EF2DFDEE3CFC74018C0686
:10159E008D071254688E298F2AAC27AD28EDD3946F
:1015AE0088EC941340031204BDE537B4241274037F
:1015BE00900050F0D2229000C5E0B402031204BD98
:1015CE00AE2BAF2CAC27AD28EF2DFDEE3CFC8C2BBB
:1015DE008D2CAE27AF28EFD39DEE9C4011900018B6
:1015EE00E0FAA3E0FBEBC394E8EA94034002800622
:1015FE00900018125484900014E0FEA3E0FFAC2774
:10160E00AD28EF2DFDEE3CFC900014ECF0A3EDF0B8
:10161E009000C5E0B4021DAE27AF287405125476B3
:10162E0074038E048F05FF125458900010ECF0A333
:10163E00EDF08016AE27AF287403125476740112A3
:10164E005468900010EEF0A3EFF0C28E758D007509
:10165E008B00753D00752801752700D28EE5372465
:10166E000875F00984AFF07E00EF4E70759000148F
:10167E00E0F8A3E0900012C8F0A3C8F0900012E0CA
:10168E00FEA3E0FFEF4E600B7C807D0E1253568E54
:10169E00258F26900014E4F0A3F0AE25AF26742813
:1016AE00BE00039F5010E53C2FFF50010E74011237
:1016BE0054688E258F2685263C9000CCE0A825B850
:1016CE00000DD395264008E52690004DF080099038
:1016DE0000CCE01490004DF0E549600675260075CB
:1016EE0025009000C3E0B40308900040E065376029
:1016FE0002802AA220B34004D2218002B22190009F
:10170E0090E0600FE549700BA220B35006A221B302
:10171E00B3400280067405900050F0C220E5376495
:10172E000B6005E537B41D099000B5E06003124962
:10173E00E8900049E06537600790004AE0B537034E
:10174E00754B00A20EB35006A20DB3B340030218A0
:10175E0088900081E0B4015AE54075F00584FF7E63
:10176E000090057B12549DE0F534753300AE33AF17
:10177E003490007FE012547674648E048F05FF124D
:10178E00545874C18C068D071254768E358F369050
:10179E000016E0FEA3E0FFAC33AD34120003746418
:1017AE008E048F05FF125458900016ECF0A3EDF046
:1017BE00800F90007FE075F0C1A4FFAEF08E358FE4
:1017CE0036E53AC394CC500690007FE070030218C1
:1017DE008685F95085FA517E017F00E551125476C7
:1017EE00E5502FFF50010E8E338F34AC35AD36EFF2
:1017FE002DFDEE3CFC8C358D36E536F5FBE535F5ED
:10180E00FCE536F5E9E535F5EAE536F5EBE535F5D2
:10181E00ECE536F5EDE535F5EED293D294D291D2D4
:10182E00929000C3E0B4035075A71085F95085FA65
:10183E00517E017F00E551125476E5502FFF500185
:10184E000E8E338F34E536F5FBE535F5FCE536F5D2
:10185E00E9E535F5EAE536F5EBE535F5ECE536F592
:10186E00EDE535F5EED287D290E5B54410F5B5E548
:10187E00B54420F5B575A700D20EE549B40106E5CD
:10188E0037640B6002800F754C019000537401F0A9
:10189E00E5B54401F5B5E54960030219489000C865
:1018AE00E0600D9000CFE0A825B800069526400216
:1018BE0080429000C8E0B4022790003CE06537609B
:1018CE001790003DE06537600F90003EE065376091
:1018DE000790003FE0B53703754C03754500800C4B
:1018EE00C20075450090001EE4F0A3F0740990004C
:1018FE0050F0804690003CE0B5370B754C019000DF
:10190E00537401F0803490003DE0B5370B754C01F7
:10191E007402900053F0802290003EE0B5370B75B4
:10192E004C017403900053F0801090003FE0B537E7
:10193E0009754C017404900053F0A20BB39209A2E6
:10194E000BB330B601B35003021A36754A0190003C
:10195E00A8E07013A20BB34008E5B54404F5B580BA
:10196E0006E5B554FBF5B5A20B9209E537D3944ABB
:10197E004014D20DE537D3946E400B740390005093
:10198E00F0D2227537469000D0E0B40107E543C38C
:10199E009414400280031204BD7446900073F0A2AA
:1019AE0004300501B35017A204B34008E5B544084E
:1019BE00F5B58006E5B554F7F5B5A2049205A20675
:1019CE00300701B35017A206B34008E5B54402F53F
:1019DE00B58006E5B554FDF5B5A2069207E543C3FD
:1019EE0094415009740E900050F01204BD90005AAC
:1019FE00E0FE900056E004C39E4009900056E0D3EE
:101A0E009406400974FB900050F01204BD90005FE4
:101A1E00E0601590005FE0FE900059E06E60097482
:101A2E00FE900050F01204BDA222B34008C296C22E
:101A3E0095C2A0C297A210B3B35008900040E065C3
:101A4E00376003021B2FA202B35006A200B3B340AD
:101A5E0003021B279000C3E0B40370A208B3403901
:101A6E00A221B3400F12009EE536F5FBE535F5FCDD
:101A7E00D29380101200CBE536F5FBE535F5FCD29E
:101A8E008775A700A203B34008E5B54440F5B580BD
:101A9E0006E5B554BFF5B5803012009EE536F5FB70
:101AAE00E535F5FCD2931200CBE536F5FBE535F5C1
:101ABE00FCD28775A700A203B34008E5B54440F5F4
:101ACE00B58006E5B554BFF5B5804E9000E1E0C394
:101ADE009402501612009EE536F5FBE535F5FCD264
:101AEE0093A203B34002D287802F12009EE536F5F3
:101AFE00FBE535F5FCD2931200CBAE33AF34AC56CA
:101B0E00AD57EF2DFDEE3CFC8C358D36E536F5FBF5
:101B1E00E535F5FCD28775A700C210D211D212D2CC
:101B2E0013A211B3B35008900041E0653760030271
:101B3E001C1BA202B35006A200B3B34003021C1337
:101B4E009000C3E0B40370A208B34039A221B340A1
:101B5E000F12009EE536F5E9E535F5EAD2948010D0
:101B6E001200CBE536F5E9E535F5EAD29075A7001A
:101B7E00A203B34008E5B54440F5B58006E5B5547B
:101B8E00BFF5B5803012009EE536F5E9E535F5EA8C
:101B9E00D2941200CBE536F5E9E535F5EAD290752B
:101BAE00A700A203B34008E5B54440F5B58006E5AD
:101BBE00B554BFF5B5804E9000E1E0C394025016C7
:101BCE0012009EE536F5E9E535F5EAD294A203B3A7
:101BDE004002D290802F12009EE536F5E9E535F5EC
:101BEE00EAD2941200CBAE33AF34AC56AD57EF2DD4
:101BFE00FDEE3CFC8C358D36E536F5E9E535F5EA3E
:101C0E00D29075A700D210C211D212D213A212B363
:101C1E00B35008900042E065376003021D17A20220
:101C2E00B35006A200B3B34003021D0F9000C3E0F1
:101C3E00B40378A208B3403DA221B3400F12009E18
:101C4E00E536F5EBE535F5ECD29180141200CBE5D7
:101C5E0036F5EBE535F5ECE5B54410F5B575A700B1
:101C6E00A203B34008E5B54440F5B58006E5B5548A
:101C7E00BFF5B5803412009EE536F5EBE535F5EC93
:101C8E00D2911200CBE536F5EBE535F5ECE5B54432
:101C9E0010F5B575A700A203B34008E5B54440F5AD
:101CAE00B58006E5B554BFF5B580569000E1E0C3AA
:101CBE009402501A12009EE536F5EBE535F5ECD29E
:101CCE0091A203B34006E5B54410F5B5803312007A
:101CDE009EE536F5EBE535F5ECD2911200CBAE3341
:101CEE00AF34AC56AD57EF2DFDEE3CFC8C358D363A
:101CFE00E536F5EBE535F5ECE5B54410F5B575A72C
:101D0E0000D210D211C212D213A213B3B350089044
:101D1E000043E065376003021E13A202B35006A211
:101D2E0000B3B34003021E0B9000C3E0B40378A2CD
:101D3E0008B3403DA221B3400F12009EE536F5EDEB
:101D4E00E535F5EED29280141200CBE536F5EDE5D1
:101D5E0035F5EEE5B54420F5B575A700A203B34001
:101D6E0008E5B54440F5B58006E5B554BFF5B58038
:101D7E003412009EE536F5EDE535F5EED292120001
:101D8E00CBE536F5EDE535F5EEE5B54420F5B57563
:101D9E00A700A203B34008E5B54440F5B58006E5BB
:101DAE00B554BFF5B580569000E1E0C39402501AC9
:101DBE0012009EE536F5EDE535F5EED292A203B3AF
:101DCE004006E5B54420F5B5803312009EE536F5A4
:101DDE00EDE535F5EED2921200CBAE33AF34AC5604
:101DEE00AD57EF2DFDEE3CFC8C358D36E536F5ED21
:101DFE00E535F5EEE5B54420F5B575A700D210D260
:101E0E0011D212C213E54CB4081A124317A210B322
:101E1E005005A211B340028008D210D211D212D2B4
:101E2E0013754C1EE54CB407061240CF754C08E5F1
:101E3E004CB4063D900016E0FEA3E0FFEF4E6006A8
:101E4E00A208B3B340028023AE52AF53900016E007
:101E5E00FCA3E0FDEF2DFDEE3CFC8C528D53E537DF
:101E6E00D394095006900016120039123EA1754CFB
:101E7E0007E54CB40506123D01754C06E54CB4045D
:101E8E00329000B6E0903388F82828731239958086
:101E9E0012123995800D123B438008123BF58003D8
:031EAE00123BF5EF
:0F338800021E9A021E9F021EA4021EA9021EAE62
:101EB100900098E06005124AD18002C204754C0579
:101EC100E54CB403028003021FAB90009BE0600568
:101ED100124BDE8002C2069000B6E0D39402403F6E
:101EE10090008AE02403A825B800049526500990A3
:101EF100008CE0D3953A50028008D2027408900019
:101F010050F090008AE0A825B80005D39526500B23
:101F110090008CE02403C3953A5002C202803990AC
:101F2100008AE02403A825B8000495265007E53867
:101F3100C3953940028008D2027408900050F09095
:101F4100008AE0A825B80005D395265009E5392473
:101F51000FC395385002C2029000D0E07007E543EC
:101F6100C3941440028002D202A2024005754C04BF
:101F7100800A754C1E90001EE4F0A3F0A208B34045
:101F810029E54075F00584FF7E0090057B12549D84
:101F9100E0C394695005124A1D800F9007B5E0F81F
:101FA100A3E09007B3C8F0A3C8F0E54CB40A0280DF
:101FB1000302204990002EE0C394465008C2967453
:101FC1004690002EF0900044E0B4011DE55A240A29
:101FD100F55A9007B7E0FEA3E0FF740A2FFF500106
:101FE1000E9007B7EEF0A3EFF0855A3475330090E9
:101FF100003CE0F5501200FBE53690002EF0900019
:1020010008E533F0A3E534F0E55090002FF0C21558
:102011009007B7E0F533A3E0F53490003CE0F550CC
:102021001200FBE53690002CF0900000E533F0A3A0
:10203100E534F0E55090002DF0C214E549B40105F6
:10204100754C0B8003754C0390002CE0B53773A2DF
:1020510014404F900000E0FEA3E0FFEF4E6021AE80
:1020610029AF2A900000E0FCA3E0FD120003740AEE
:102071008E048F05FF125458900000ECF0A3EDF090
:1020810090002DE0601A900000E0FEA3E0FFAC2973
:10209100AD2AEF2DFDEE3CFC900000ECF0A3EDF03D
:1020A100D214AE27AF28900000E0FCA3E0FDEFC3FF
:1020B1009DEE9C400D120591D296C21474C89000F9
:1020C1002CF0A214B3B3500790002CE0B537028076
:1020D1000D120591D29674C890002CF0C214900094
:1020E1002EE0B53770A215404F900008E0FEA3E046
:1020F100FFEF4E6021AE29AF2A900008E0FCA3E07B
:10210100FD120003740A8E048F05FF1254589000CB
:1021110008ECF0A3EDF090002FE0601A900008E0C9
:10212100FEA3E0FFAC29AD2AEF2DFDEE3CFC9000B3
:1021310008ECF0A3EDF0D215AE27AF28900008E02F
:10214100FCA3E0FDEFC39DEE9C400AC2967446904D
:10215100002EF0C215A215B3B3500790002EE0B5C2
:102161003702800AC296744690002EF0C215E54CE3
:10217100B40B028003022218900032E0C39446504F
:10218100139000D1E0B40104C2968002C295744656
:10219100900032F0900045E0B4011DE55A240AF5A3
:1021A1005A9007B7E0FEA3E0FF740A2FFF50010E1B
:1021B1009007B7EEF0A3EFF0855A34753300900025
:1021C1003DE0F5501200FBE536900032F090000A38
:1021D100E533F0A3E534F0E550900033F0C21790F9
:1021E10007B7E0F533A3E0F53490003DE0F5501278
:1021F10000FBE536900030F0900002E533F0A3E5F6
:1022010034F0E550900031F0C216E549B40105758E
:102211004C0C8003754C03900030E0B5377EA2165C
:10222100404F900002E0FEA3E0FFEF4E6021AE2997
:10223100AF2A900002E0FCA3E0FD120003740A8EB5
:10224100048F05FF125458900002ECF0A3EDF090BA
:102251000031E0601A900002E0FEA3E0FFAC29AD7E
:102261002AEF2DFDEE3CFC900002ECF0A3EDF0D244
:1022710016AE27AF28900002E0FCA3E0FDEFC39D5E
:10228100EE9C40181205919000D1E0B40104D29661
:102291008002D295C21674C8900030F0A216B3B372
:1022A1005007900030E0B537028018120591900078
:1022B100D1E0B40104D2968002D29574C890003066
:1022C100F0C216900032E0B5377BA217404F900064
:1022D1000AE0FEA3E0FFEF4E6021AE29AF2A900095
:1022E1000AE0FCA3E0FD120003740A8E048F05FFCF
:1022F10012545890000AECF0A3EDF0900033E06026
:102301001A90000AE0FEA3E0FFAC29AD2AEF2DFDF3
:10231100EE3CFC90000AECF0A3EDF0D217AE27AF33
:102321002890000AE0FCA3E0FDEFC39DEE9C401560
:102331009000D1E0B40104C2968002C29574469027
:102341000032F0C217A217B3B35007900032E0B5C4
:10235100370280159000D1E0B40104C2968002C218
:10236100957446900032F0C217E54CB40C0280031C
:10237100022413900036E0C3944650139000D1E03C
:10238100B40104C2968002C2A07446900036F09057
:102391000046E0B4011DE55A240AF55A9007B7E05A
:1023A100FEA3E0FF740A2FFF50010E9007B7EEF075
:1023B100A3EFF0855A3475330090003EE0F55012DA
:1023C10000FBE536900036F090000CE533F0A3E514
:1023D10034F0E550900037F0C2199007B7E0F533BB
:1023E100A3E0F53490003EE0F5501200FBE5369095
:1023F1000034F0900004E533F0A3E534F0E55090AB
:102401000035F0C218E549B40105754C0D8003751E
:102411004C03900034E0B5377EA218404F90000481
:10242100E0FEA3E0FFEF4E6021AE29AF2A90000449
:10243100E0FCA3E0FD120003740A8E048F05FF1275
:102441005458900004ECF0A3EDF0900035E0601AD0
:10245100900004E0FEA3E0FFAC29AD2AEF2DFDEED4
:102461003CFC900004ECF0A3EDF0D218AE27AF28AD
:10247100900004E0FCA3E0FDEFC39DEE9C40181228
:1024810005919000D1E0B40104D2968002D2A0C29D
:102491001874C8900034F0A218B3B35007900034F8
:1024A100E0B5370280181205919000D1E0B4010423
:1024B100D2968002D2A074C8900034F0C218900065
:1024C10036E0B5377BA219404F90000CE0FEA3E047
:1024D100FFEF4E6021AE29AF2A90000CE0FCA3E093
:1024E100FD120003740A8E048F05FF1254589000E8
:1024F1000CECF0A3EDF0900037E0601A90000CE0D6
:10250100FEA3E0FFAC29AD2AEF2DFDEE3CFC9000CF
:102511000CECF0A3EDF0D219AE27AF2890000CE03F
:10252100FCA3E0FDEFC39DEE9C40159000D1E0B40B
:102531000104C2968002C2A07446900036F0C2190E
:10254100A219B3B35007900036E0B5370280159059
:1025510000D1E0B40104C2968002C2A0744690008A
:1025610036F0C219E54CB40D02800302260C90002E
:102571003AE0C3944650139000D1E0B40104C296EE
:102581008002C297744690003AF0900047E0B4018F
:102591001DE55A240AF55A9007B7E0FEA3E0FF743F
:1025A1000A2FFF50010E9007B7EEF0A3EFF0855A06
:1025B1003475330090003FE0F5501200FBE5369092
:1025C100003AF090000EE533F0A3E534F0E55090C9
:1025D100003BF0C21B9007B7E0F533A3E0F5349060
:1025E100003FE0F5501200FBE536900038F0900016
:1025F10006E533F0A3E534F0E550900039F0C21A56
:10260100E549B40103754900754C03900038E0B504
:10261100377EA21A404F900006E0FEA3E0FFEF4E86
:102621006021AE29AF2A900006E0FCA3E0FD120074
:1026310003740A8E048F05FF125458900006ECF0C3
:10264100A3EDF0900039E0601A900006E0FEA3E0EF
:10265100FFAC29AD2AEF2DFDEE3CFC900006ECF01D
:10266100A3EDF0D21AAE27AF28900006E0FCA3E05C
:10267100FDEFC39DEE9C40181205919000D1E0B48E
:102681000104D2968002D297C21A74C8900038F021
:10269100A21AB3B35007900038E0B5370280181280
:1026A10005919000D1E0B40104D2968002D29774D2
:1026B100C8900038F0C21A90003AE0B5377BA21BEF
:1026C100404F90000EE0FEA3E0FFEF4E6021AE29E7
:1026D100AF2A90000EE0FCA3E0FD120003740A8E05
:1026E100048F05FF12545890000EECF0A3EDF0900A
:1026F100003BE0601A90000EE0FEA3E0FFAC29ADC4
:102701002AEF2DFDEE3CFC90000EECF0A3EDF0D293
:102711001BAE27AF2890000EE0FCA3E0FDEFC39DA8
:10272100EE9C40159000D1E0B40104C2968002C233
:1027310097744690003AF0C21BA21BB3B3500790A6
:10274100003AE0B5370280159000D1E0B40104C22F
:10275100968002C297744690003AF0C21BE54CB4D1
:10276100020280030228181247801248979007B38B
:10277100E0FEA3E0FF740A125476900012E0FCA37D
:10278100E0FD74098F02FF1254588D078C038E04EB
:102791008A058B061253569007B7EEF0A3EFF0901F
:1027A10000D1E0B40108743CBE00059F4002800DD9
:1027B100743C9007B7F8E4F0E8A3F0801B9007B7EA
:1027C100E0FEA3E0FF74F0BE00039F500B74F09095
:1027D10007B7F8E4F0E8A3F09007B7E0FEA3E0FF45
:1027E100E55A2FFF50010E9007B7EEF0A3EFF090DE
:1027F1000053E0B40103754C0A900053E0B40203A6
:10280100754C0B900053E0B40303754C0C900053CE
:10281100E0B40403754C0DE54CB401259000E8E0EB
:10282100903397F828287312451E801212451E8096
:0E2831000D1245A8800812465480031246542A
:0F33970002282802282D02283202283702283C5B
:10283F00754C029000D3E0B40202800302295A9033
:10284F000076E0D3953F5064900076E0F404253F86
:10285F00FE9000D6E08E00F5F0E884FF7E008F50EA
:10286F00EFC39410500CEF8550F0A4FDACF08D50D9
:10287F0080037550FF900076E0D39550400B900089
:10288F0076E0C39550F54D8003754D009000F1E053
:10289F00D3954D40069000F1E0F54D9000F2E0C366
:1028AF00954D50069000F2E0F54D8071900076E066
:1028BF00C3953FFE9000D6E08E00F5F0E884FF7ED2
:1028CF00008F50EFC39410500CEF8550F0A4FDAC67
:1028DF00F08D5080037550FF855034753300900094
:1028EF0076E02534FFAE3350010E8E338F3474FFF4
:1028FF00BE0009D39F400585344D8003754DFF9071
:10290F0000F1E0D3954D40069000F1E0F54D9000B9
:10291F00F2E0C3954D50069000F2E0F54DA208B3DA
:10292F00B350099000DEE0D3954E5002800A740731
:10293F00900050F0C2A2801375A710E5CDC3954D3E
:10294F004004C2A28002D2A275A700E54BC394092E
:10295F004003023095A2EDB35003023095C2EDE56E
:10296F004B6003022B09900084E07003022AF89059
:10297F0000BAE0B401028003022A58900049E0B582
:10298F0037028003022A557E017F00E5BE1254767E
:10299F00E5BD2FFF50010E8E338F34900084E0B4CD
:1029AF000118741012547690007AE08E048F05FF90
:1029BF00125458ED90004BF0802CAE33AF3474109E
:1029CF0012547690007AE08E048F05FF12545890BF
:1029DF00004BE02DFD50010C74018C068D07125435
:1029EF0068EF90004BF0E54460089000E0E064026F
:1029FF00600280219000E2E0B4011A90004BE07574
:102A0F00F0E7A4FFAEF0E5448E048F05FF12545893
:102A1F00ED90004BF090004BE0FE90004CE0D39E09
:102A2F004004D21E8002B21E90004BE090004CF08A
:102A3F009000B6E064016006A21EB3B340028006A8
:102A4F0090004BE0F538022AF6D21E7E017F00E59A
:102A5F00BE125476E5BD2FFF50010E8E338F34908A
:102A6F000084E0B40118741012547690007AE08E4E
:102A7F00048F05FF125458ED90004BF0802CAE33AD
:102A8F00AF34741012547690007AE08E048F05FFE5
:102A9F0012545890004BE02DFD50010C74018C0620
:102AAF008D07125468EF90004BF0E54460089000DA
:102ABF00E0E06402600280219000E2E0B4011A902D
:102ACF00004BE075F0E7A4FFAEF0E5448E048F05F0
:102ADF00FF125458ED90004BF09000B6E064016087
:102AEF000690004BE0F5388003753800900080E0C9
:102AFF007005754B01800375BB18E54BB40102805F
:102B0F0003022CAB900080E07003022C9A7E017FB1
:102B1F0000E5BE125476E5BD2FFF50010E8E338FA8
:102B2F00349000C6E0B4010F7E0F7FFFAC33AD349D
:102B3F001254CB8E338F349000EBE0B40245AE339A
:102B4F00AF34900028E0FCA3E0FDEDD39FEC9E4056
:102B5F000A900028E533F0A3E534F0AE33AF34909C
:102B6F00002AE0FCA3E0FDEFD39DEE9C400A90000D
:102B7F002AE533F0A3E534F0AE33AF3474041254C6
:102B8F00688F3A9000EBE0704CAE33AF3490002872
:102B9F00E0FCA3E0FDEFD39DEE9C40091254CB8ED9
:102BAF00338F348006753400753300AE33AF347411
:102BBF0010125476900077E08E048F05FF12545850
:102BCF008C338D347400D39D74019C400585343A49
:102BDF008003753AFF9000B6E0B401028003022C27
:102BEF0098A208B3B3500E90008AE0A825B800054C
:102BFF00D395265003022C8D90008BE075F019A40D
:102C0F00FFAEF09000CEE08E048F05FF1254589067
:102C1F0000C7E0853AF0A4FFAEF074648D028C0318
:102C2F008E048F05FF125458EA2DFDEB3CFC8C33BC
:102C3F008D34E544600F9000E0E0B402089000E2AC
:102C4F00E0640160028017AE33AF3474E71254763C
:102C5F00E5448E048F05FF1254588C338D34900049
:102C6F004BE0A833B8000AD395344005853438803B
:102C7F000BA21EB3400690004BE0F538800BA21E4E
:102C8F00B3400690004BE0F5388003753A00900092
:102C9F0083E07005754B02800375BB19E54BB402D9
:102CAF00028003022D66900083E07003022D55E52C
:102CBF0037D394124003022D53900026E0FEA3E079
:102CCF00FFE53E1254C3900026EEF0A3EFF07E0115
:102CDF007F00E5BE125476E5BD2FFF50010E8E33F7
:102CEF008F349000F0E07013740A12547674518E82
:102CFF00048F05FF1254588D3E8019AE33AF3474D4
:102D0F000A1254768F048E057E017F95CDCCCD129D
:102D1F0053568F3EE53ED394644003753E64900056
:102D2F0026E0FEA3E0FFE53E2FFF50010E900026A8
:102D3F00EEF0A3EFF0900087E0048E048F05FF12F2
:102D4F0054588D3E8003753E329000D3E070057568
:102D5F004B03800375BB13E54BB4035E9000D3E0C8
:102D6F0060477E017F00E5BE125476E5BD2FFF5010
:102D7F00010E8E338F3474041254688F3F9000D538
:102D8F00E0853FF0A4FDACF07464FF1254588D3F02
:102D9F009000D4E0853FF0A4FFAEF074FF8E048F57
:102DAF0005FF1254588D4E8003753F00900081E04F
:102DBF007005754B04800375BB17E54BB404028097
:102DCF0003022E67900081E0B4017C7E017F00E555
:102DDF00BE125476E5BD2FFF50010E7404125468D5
:102DEF008E338F3490004EE0601290004EE01490BE
:102DFF00526493A833B800069534400280069000C1
:102E0F004EE014F090004EE0C39477501390004EB4
:102E1F00E00490526493A833B80005D39534500260
:102E2F00800690004EE004F090004EE0FE9000A768
:102E3F00E08E0088F0A4FFAEF074648E048F05FF5F
:102E4F001254588D408003754000900082E0700549
:102E5F00754B05800375BB16E54BB4050280030265
:102E6F002EFA900082E0B4017C7E017F00E5BE1255
:102E7F005476E5BD2FFF50010E74041254688E3343
:102E8F008F3490004FE0601290004FE0149052DDAD
:102E9F0093A833B8000695344002800690004FE0A7
:102EAF0014F090004FE0C39477501390004FE0045C
:102EBF009052DD93A833B80005D3953450028006A5
:102ECF0090004FE004F090004FE0FE9000ADE08ED8
:102EDF000088F0A4FFAEF074648E048F05FF1254C7
:102EEF00588D41800375410075BB1FE54BB4063308
:102EFF007E017F00E5BE125476E5BD2FFF50010E17
:102F0F008E338F34740912547674E68E048F05FF56
:102F1F001254588D43900089E07005754B0780035C
:102F2F0075BB15E54BB40702800302303C90008956
:102F3F00E0700302302B7E017F00E5BE125476E570
:102F4F00BD2FFF50010E8E338F3474041254688FCF
:102F5F0042900089E0B401159000DDE08542F0A4B5
:102F6F00FFAEF07407125468EF9007C0F09000891D
:102F7F00E0B402159000DDE08542F0A4FFAEF074DE
:102F8F0007125468EF9007BFF0900089E0B4030276
:102F9F0080030230299000CAE0701CE542C3940AF6
:102FAF005002D201E542D394644002C2019000A9BD
:102FBF00E0900075F080639000A9E070349000DD20
:102FCF00E08542F0A4FFAEF074FF8E048F05FF1270
:102FDF005458ED900075F0AE25AF26741EBE000656
:102FEF00D39F4002D201E53AD394E54002C201805B
:102FFF0029E542C3940A500DAE25AF26741EBE00BC
:10300F0004D39F50028002D201E53AD394E54002E7
:10301F00C2019000A9E0900075F080037542009006
:10302F0000E0E07005754B08800375BB14E54BB4E9
:10303F0008509000E0E060397E017F00E5BE125439
:10304F0076E5BD2FFF50010E8E338F34EFD39421D1
:10305F00EE940E40057544FF8015AE33AF347410F7
:10306F0012547674E38E048F05FF1254588D4480EA
:10307F0003754400900084E0600575BB1A800375EA
:10308F00BB18054BD2ECAE27AF287410C39F742723
:10309F009E400C900074E0C3943C4003023385C201
:1030AF000D7537469000C5E07005754902800375B0
:1030BF004903C293C294C291C292C287C290E5B52E
:1030CF0054EFF5B5E5B554DFF5B5C296C295C2A07C
:1030DF00C297C2A2C2A1E5B554BFF5B5E5B5547FFD
:1030EF00F5B5A21FB34008E5B54404F5B58006E574
:1030FF00B554FBF5B5A20FB3500EE53AD394334058
:10310F0007E53AC394CC4003023219E5B54401F503
:10311F00B57446900073F090007FE075F064A4FFE3
:10312F00AEF08E358F367402BE000AD39F400675FF
:10313F00360275350085F95085FA517E017F00E51D
:10314F0051125476E5502FFF50010E8E338F34AC51
:10315F0035AD36EF2DFDEE3CFC8C358D36E536F575
:10316F00FBE535F5FCE536F5E9E535F5EAE536F548
:10317F00EBE535F5ECE536F5EDE535F5EED293D229
:10318F0094D291D2929000C3E0B4037C90007FE080
:10319F0075F0BEA4FBAAF08A358B367402BA000A0A
:1031AF00D39B400675360275350075A71085F9500B
:1031BF0085FA517E017F00E551125476E5502FFFBD
:1031CF0050010E8E338F34AC35AD36EF2DFDEE3C06
:1031DF00FC8C358D36E536F5FBE535F5FCE536F53A
:1031EF00E9E535F5EAE536F5EBE535F5ECE536F5E8
:1031FF00EDE535F5EED287D290E5B54410F5B5E59E
:10320F00B54420F5B575A700D20FE53AC3941A500F
:10321F0002C20F90001074FFF0A374DCF09000A6B0
:10322F00E0900016F8E4F0E8A3F0C214C216C2183A
:10323F00C21A74C890002CF074C8900030F074C893
:10324F00900034F074C8900038F0C210C211C2124E
:10325F00C213752600752500753C00C208756C00F9
:10326F0090001EE4F0A3F0754C1E9007B5E0FEA38E
:10327F00E0FF740312547674011254689007B3EE92
:10328F00F0A3EFF0900098E06005124AD18002C2DF
:10329F000490009BE06005124BDE8002C206A20480
:1032AF00300501B35017A204B34008E5B54408F543
:1032BF00B58006E5B554F7F5B5A2049205A2063020
:1032CF000701B35017A206B34008E5B54402F5B5A0
:1032DF008006E5B554FDF5B5A2069207C203752C1D
:1032EF0000752B00900018E4F0A3F0900087E075B4
:1032FF00F032A4FFAEF0900026EEF0A3EFF09000B6
:10330F0014E4F0A3F0C225900074E0C3943C501075
:10331F00E54BB40909900074E004F0754B00803B55
:10332F00E54BB40903754B00752800752700758DA3
:10333F0000758B00753D00900073E0C394645008D6
:10334F00900073E004F080067464900073F09000B6
:10335F0073E0B46406E5B554FEF5B5900074E0D3A0
:10336F0094014007E543C3944140028009740E90D5
:09337F000050F01204BD020D150E
:1051EC000000010001400160018001A001C001E04C
:1051FC0002000300039603B603D603F40400050073
:10520C0005180530054805600578059005A805C00A
:10521C00060006140628063C066E068C00FF013FAD
:10522C00015F017F019F01BF01DF01FF02FF0395B9
:10523C0003B503D503F303FF04FF0517052F05473B
:10524C00055F0577058F05A705BF05FF0613062724
:10525C00063B066F068B06A9DAD8D7D5D4D2D0CFA9
:10526C00CDCBC9C7C6C4C2C0BEBCBAB8B5B3B1AF4A
:10527C00ADABA8A6A4A2A09D9B99969492908D8B61
:10528C0089878482807E7C79777573716F6D6B6989
:10529C00676563615F5D5B5957565452504F4D4B78
:1052AC004A4847454442413F3E3C3B3A3937363504
:1052BC00343231302F2E2D2C2B2A29282726252528
:1052CC002423222121201F1E1E1D1C1C1B1A1A19EF
:1052DC0019EEECEBEAE9E8E7E5E4E3E1E0DEDDDB3F
:1052EC00D9D8D6D4D2D0CECCCAC8C6C3C1BFBCBA0A
:1052FC00B7B5B2B0ADABA8A5A3A09D9B9895929065
:10530C008D8A8785827F7D7A7775726F6D6A686505
:10531C0063615E5C5A575553514F4D4B494745435A
:10532C0042403E3C3B393836353332312F2E2D2B13
:10533C002A292827262524232221201F1E1D1D1C37
:0A534C001B1A1A1918181716161567
:1033A600750B00750A00AE0AAF0BAC08AD09EDC38C
:1033B6009FEC9E401674FF12544875CF01780B742B
:1033C6000126F6500418E436F650DB22900048E059
:1033D600B4AA1C90077BE0B43C159007BBE0FEA3A3
:1033E600E0FFEF4E6009741EBE0004D39F50030237
:1033F600350075360075350075F8099007BBE0FE97
:10340600A3E0FF74076F4E6006740E6F4E7006746D
:103416003A90077BF09007BBE0FEA3E0FF7408BE7E
:10342600001ED39F401A7E017F089007BBE0FCA3D5
:10343600E0FD1DBDFF011C1200038E338F34801F7B
:103446009007BBE0FEA3E0FF74081254C38F048EFE
:10345600057E017F08CDCCCD1200038E338F34AEAE
:1034660035AF36740CD39F74019E50030234FBA211
:10347600F9B3407EE5364535700375A382AE35AFA8
:103486003674016F4E700375A300AE35AF36740205
:103496006F4E700D9007BCE075F002A4FDACF08D88
:1034A600A3AE35AF3674036F4E700375A300AE3509
:1034B600AF367403BE00039F5013AC33AD34ED2F0B
:1034C600FFEC3EFE90007712549DE0F5A3AE35AFBB
:1034D60036EFB40B09EEB401057414125448AE3538
:1034E600AF36EFB40B07EEB4010375F80D7835125D
:1034F60054D3023465900048E4F0227536007535E1
:103506000075F8099007BBE0FEA3E0FF7408BE0053
:103516001ED39F401A7E017F089007BBE0FCA3E004
:10352600FD1DBDFF011C1200038E338F34801F90DA
:1035360007BBE0FEA3E0FF74081254C38F048E0598
:103546007E017F08CDCCCD1200038E338F34AE358D
:10355600AF367411D39F74019E5003023631A2F91F
:10356600B3500302362EE5364535700375A3D2AE49
:1035760035AF3674016F4E700375A300AE35AF36A6
:1035860074026F4E700D9007BCE075F002A4FDAC9E
:10359600F08DA3AE35AF3674036F4E700375A3007E
:1035A600AE35AF3674046F4E700375A300AE35AFFB
:1035B6003674056F4E700375A300AE35AF367406CC
:1035C6006F4E700375A300AE35AF3674076F4E703D
:1035D6000375A300AE35AF3674086F4E700375A33E
:1035E60000AE35AF367408BE00039F5016AC33AD3F
:1035F60034ED2FFFEC3EFE90007212549DE5A3F0D1
:1036060075A300AE35AF36EFB41009EEB4010574FC
:1036160014125448AE35AF36EFB41007EEB40103BA
:1036260075F80D78351254D3023554227536007567
:10363600350075F809AE35AF367417BE0004D39F52
:10364600500302370AA2F9B35003023707E536459D
:1036560035700375A3D2AE35AF3674016F4E700365
:1036660075A300AE35AF3674026F4E700D9007BC71
:10367600E075F002A4FDACF08DA3AE35AF36740351
:103686006F4E700375A300AE35AF3674046F4E707F
:103696000375A300AE35AF3674056F4E700375A380
:1036A60000AE35AF3674066F4E700375A300AE35A7
:1036B600AF3674076F4E700375A300AE35AF367420
:1036C600086F4E700375A300AE35AF367408BE00A2
:1036D600039F500C90005C12549DE5A3F075A30067
:1036E600AE35AF3674166F4E70057414125448AE6C
:1036F60035AF3674166F4E700375F80D7835125463
:10370600D302363B22900048E0B4AB028003023776
:10371600A575360075350075F809AE35AF367412E5
:10372600BE007CD39F4078A2F9B34070E53645359C
:10373600700375A382AE35AF3674016F4E70037594
:10374600A300AE35AF3674026F4E700D9007BCE025
:1037560075F002A4FDACF08DA3AE35AF3674036FE1
:103766004E700375A300AE35AF367403BE00039FDB
:10377600500990006112549DE0F5A3AE35AF367442
:10378600116F4E70057414125448AE35AF3674116D
:103796006F4E700375F80D78351254D30237202218
:1037A600900051E4F074649007BBF8E4F0E8A3F0ED
:1037B60012363274C89007BBF8E4F0E8A3F0900024
:1037C60068E0B4371A900065E090005CF0900066FF
:1037D600E090005DF0900067E090005EF08046901B
:1037E60000517401F074659007BBF8E4F0E8A3F0AB
:1037F60012363274C89007BBF8E4F0E8A3F09000E4
:1038060068E0B4371A900065E090005CF0900066BE
:10381600E090005DF0900067E090005EF080067436
:1038260002900051F0900052E4F074669007BBF8E5
:10383600E4F0E8A3F012363274C89007BBF8E4F05F
:10384600E8A3F0900067E0B43712900065E09000BE
:1038560056F0900066E090005FF08076900052741B
:1038660001F074679007BBF8E4F0E8A3F012363273
:1038760074C89007BBF8E4F0E8A3F0900067E0B4E2
:103886003712900065E0900056F0900066E09000D8
:103896005FF0803E7402900052F074689007BBF8A7
:1038A600E4F0E8A3F012363274C89007BBF8E4F0EF
:1038B600E8A3F0900067E0B43712900065E090004E
:1038C60056F0900066E090005FF08006740390006A
:1038D60052F022E55D2534FFAE3350010E90007B99
:1038E60012549DE0F55EE55D2534FFAE3350010EC2
:1038F6000FBF00010E90007B12549DE0F55F8565B9
:1039060061E55EB55F05855E5D8041E55FD3955EE9
:10391600401DE55FC3955E8560F0A4FFAEF0E561EE
:103926008E048F05FF125458ED255EF55D801DE56A
:103936005EC3955F8560F0A4FFAEF0E5618E048FEF
:1039460005FF125458EDF404255EF55D22E55FD3BC
:10395600955E401DE55FC3955E8560F0A4FFAEF001
:10396600E5618E048F05FF125458ED255EF55D80E6
:103976001DE55EC3955F8560F0A4FFAEF0E5618E40
:10398600048F05FF125458EDF404255EF55D22E51B
:103996003875F00484FF7E008F5DE53875F0048489
:1039A600ADF07C008D60756504753301753400E5F6
:1039B6005DC3943F50051238D980069001BAE0F5F0
:1039C6005D855D5375520090004DE075F020A4FFB3
:1039D600AEF09000CCE08E048F05FF1254588D5D3A
:1039E6009000B4E0D395385003023A9B9000D8E09B
:1039F600D395384010ED9001BB1254A8E0F55575EB
:103A06005400023A989000A3E0D395384043E55D10
:103A16009001BB1254A8E0F55EE55D9001DB1254FF
:103A2600A8E0F55F9000D8E0F4042538F560900032
:103A3600A3E0FE9000D8E0F4042EF561E55EB55FE4
:103A460005855E5D8003123953855D55755400808A
:103A560041E55D9001DB1254A8E0F55EE55D90015D
:103A6600FB1254A8E0F55F9000A3E0F4042538F5B6
:103A7600609000B4E0FE9000A3E0F4042EF561E54A
:103A86005EB55F05855E5D8003123953855D5575AC
:103A96005400023B429000DBE0D395385011E55DBF
:103AA60090023B1254A8E0F555755400023B429033
:103AB60000A4E0D395385043E55D90021B1254A84C
:103AC600E0F55EE55D90023B1254A8E0F55F9000DC
:103AD600A4E0F4042538F5609000DBE0FE9000A435
:103AE600E0F4042EF561E55EB55F05855E5D800355
:103AF600123953855D557554008041E55D9001FB93
:103B06001254A8E0F55EE55D90021B1254A8E0F59C
:103B16005F9000B4E0F4042538F5609000A4E0FE60
:103B26009000B4E0F4042EF561E55EB55F05855EB0
:103B36005D8003123953855D55755400229000EC63
:103B4600E0F562756511753302753400AE25AF2652
:103B5600E56275F00FA4FDACF0EDD39FEC9E40211D
:103B6600E5628E048F05FF125458ED75F010A4FF20
:103B7600AEF0E53875F01184FD7C00ED2FF563801D
:103B86000EE53875F01184FF7E00EF24F0F56385AD
:103B9600635DE53875F01184AFF07E008F601238F2
:103BA600D9855D64AE25AF269000ECE075F00FA4D4
:103BB600FDACF0EDD39FEC9E4028753302753410B2
:103BC60085635D1238D985645E855D5FAE25AF2657
:103BD600E5628E048F05FF1254918D608562611235
:103BE6003953855D5375520075556475540022909E
:103BF60000ECE0F562756511753302753400AE258B
:103C0600AF26E56275F00FA4FDACF0EDD39FEC9EF8
:103C16004021E5628E048F05FF125458ED75F010B1
:103C2600A4FFAEF0E53A75F01184FD7C00ED2FF5AA
:103C360063800EE53A75F01184FF7E00EF24F0F5FF
:103C46006385635DE53A75F01184AFF07E008F60A1
:103C56001238D9855D64AE25AF269000ECE075F08C
:103C66000FA4FDACF0EDD39FEC9E40287533027592
:103C7600341085635D1238D985645E855D5FAE2537
:103C8600AF26E5628E048F05FF1254918D60856222
:103C960061123953855D537552009000B6E0B40445
:103CA60053E53875F00484FF7E008F5DE53875F0C6
:103CB6000484ADF07C008D60756504753301753440
:103CC60000E55DC3943F50051238D980069001BACD
:103CD600E0F55DAE52AF53E55D12547674648E0422
:103CE6008F05FF125458AE52AF53EF2DFDEE3CFC3C
:103CF6008C528D5375556475540022900081E0B442
:103D06000146E54075F00584FF7E008F5DE5407550
:103D1600F00584ADF07C008D60756505753305751D
:103D26003400E55DC3941750051238D98006900516
:103D360092E0F55DAE54AF55E55D2FFF50010E7470
:103D4600641254C38E548F55900082E0B40146E548
:103D56004175F00584FF7E008F5DE54175F00584B1
:103D6600ADF07C008D60756505753305753448E5E5
:103D76005DC3941750051238D980069005DAE0F530
:103D86005DAE54AF55E55D2FFF50010E74641254BD
:103D9600C38E548F55900091E0B40249E543C39415
:103DA6004175F00584FF7E008F5DE54375F005845F
:103DB600ADF07C008D60756505753306753400E5DC
:103DC6005DC3941350051238D9800690068EE0F52F
:103DD6005DAE54AF55E55D2FFF50010E746412546D
:103DE600C38E548F559000D3E0B402028003023E86
:103DF600A0E53875F01584FF7E008F5DE53875F017
:103E06001584ADF07C008D607565157533037534CA
:103E1600F4E55DC3940B50051238D9800690047AF8
:103E2600E0F55DE55D75F0FFA4FFAEF09000D4E02F
:103E36008E048F05FF125458ED900076F0E53F751D
:103E4600F078A4FFAEF074FF8E048F05FF1254586D
:103E56008C338D3474028C068D071254688F5DACDA
:103E660033AD347404FF1254918D60756504753357
:103E76000675346EE55DC3941D50051238D980066B
:103E8600900706E0F55DAE54AF55E55D2FFF500196
:103E96000E74641254C38E548F5522900089E0B478
:103EA60001179007C0E02555FFAE5450010E900053
:103EB600DDE01254C38E548F55900089E0B403168A
:103EC600A201B3B35010900075E0C39405A825B8BD
:103ED60000069526400280109000ABE02555FFAE07
:103EE6005450010E8E548F55900083E0B402028028
:103EF600030240CE900086E0602FE540D3941E403A
:103F060028900018E0FEA3E0FF9000C1E075F003E2
:103F1600A4FDACF0EFD39DEE9C400E9000E5E0A82A
:103F260025B80005D3952650030240CE9000CEE07A
:103F36008538F0A4FFAEF074051254767407125457
:103F4600688E338F3490008DE0A825B8000495263E
:103F5600501290008EE075F002A4FDACF0EFC39D08
:103F6600EE9C40030240CEE53875F00B84FF7E00E0
:103F760090060B12549DFEE0FFEE900085E0FEEFEA
:103F86008E0088F0A4FFAEF074648E048F05FF12D5
:103F960054588C338D3490004DE075F018A4FFAE64
:103FA600F09000CCE08E048F05FF1254588C068DDD
:103FB6000790062312549DAE33AF34E01254767444
:103FC600648E048F05FF1254588C338D34E53EA859
:103FD60033B80077D395344072E53EC39534FFE499
:103FE6009533FE8E338F347428BE00039F500C75B4
:103FF6003428753300740D900050F0AE33AF349012
:104006000086E012547674288E048F05FF125458E9
:104016008C338D34AE52AF53740A8E048F05FF1263
:1040260054588D068C07AC33AD34CFCECF12000377
:10403600740A8E048F05FF1254588C338D34AE5299
:10404600AF531254CB8E528F53807DE53EA833B8C2
:10405600000495345072AE33AF34E53E1254C38E2D
:10406600338F347428BE00039F500C753428753383
:1040760000740D900050F0AE33AF34900086E0121D
:10408600547674288E048F05FF1254588C338D3461
:10409600AE52AF53740A8E048F05FF1254588D0624
:1040A6008C07AC33AD34CFCECF120003740A8E0426
:1040B6008F05FF1254588C338D34AE52AF53EF2D0B
:1040C600FDEE3CFC8C528D5322AE52AF53AC54AD38
:1040D6005512000374648E048F05FF1254588C52D7
:1040E6008D5390007EE08C068D0712547674648E94
:1040F600048F05FF1254588C528D53A2084017AEF8
:1041060025AF267405BE00039F5002D208E53AD3B8
:1041160094CC4002D2029000E0E0B402089000E2A3
:10412600E0640160028017AE52AF53E54412547644
:1041360074E78E048F05FF1254588C528D539000ED
:10414600A0E05402601B900097E0A825B80012D3A7
:104156009526400DA208B3B35007E53AC3949A409A
:10416600028028AE5BAF5C900095E075F002A4FD7E
:10417600ACF0EF2DFDEE3CFC74022DFD50010CE57C
:104186003ABC0007D39D4003756901853A5C755BAF
:1041960000E56970030242259000F3E0C39569408B
:1041A60070E54075F00584FF7E0090057B12549DF6
:1041B600E0F534753300AE33AF349000A5E0125409
:1041C6007674648E048F05FF1254588C358D3690A4
:1041D60000F3E004C395698C068D071254769000AF
:1041E600F3E08E048F05FF1254588C358D369000FF
:1041F60096E08C068D07125476740A8E048F05FF9E
:10420600125458AE52AF53EF2DFDEE3CFC8C528D3E
:104216005305699000F3E0C39569500375690090F2
:1042260000A0E05401601B900094E0A825B800129D
:10423600D39526400DA208B3B35007E538C394CCF6
:1042460040028025900092E075F003A4FFAEF0E5F1
:10425600662FFF50010E74032FFF50010EE538BE86
:104266000007D39F4003756A01853866E56A7003C7
:104276000243009000F4E0C3956A4070E54075F093
:104286000584FF7E0090057B12549DE0F53475335E
:1042960000AE33AF349000A5E012547674648E04F9
:1042A6008F05FF1254588C358D369000F4E004C308
:1042B600956A8C068D071254769000F4E08E048F72
:1042C60005FF1254588C358D36900093E08C068D80
:1042D60007125476740A8E048F05FF125458AE5294
:1042E600AF53EF2DFDEE3CFC8C528D53056A9000CA
:1042F600F4E0C3956A5003756A009000A5E0A852E1
:10430600B80004955350099000A5E0F55375520086
:10431600229000E1E0B401028003024422A208B325
:1043260050030244209000ACE0B40168AE52AF5393
:10433600AC25AD26120003743C8E048F05FF125483
:10434600589000BCE0BC00109D400D9000BEE0A857
:1043560052B8000495535002D203AE52AF53AC2567
:10436600AD26120003743C8E048F05FF125458903C
:1043760000BCE0C3940ABC0015D39D40119000BE5A
:10438600E0C39405A852B80005D3955350028002A5
:10439600C2038068AE52AF53AC25AD26120003743B
:1043A600788E048F05FF1254589000BCE0BC0010B4
:1043B6009D400D9000BEE0A852B8000495535004ED
:1043C600D2038038AE52AF53AC25AD26120003742B
:1043D600788E048F05FF1254589000BCE0C3940AEF
:1043E600BC0015D39D40119000BEE0C39405A852B1
:1043F600B80005D3955350028002C203A203B3400E
:1044060019AE52AF539000BDE012547674648E0418
:104416008F05FF1254588C528D538002C2039000B0
:10442600E1E0B40258E53875F00884FF7E008F5D40
:10443600E53875F00884ADF07C008D60756508750B
:1044460033017534E0E55DC3943F50051238D980D9
:104456000690027AE0F55DE55D75F05EA4FFAEF0CC
:10446600740A8E048F05FF1254588C568D577402A9
:10447600BC000AD39D4006755702755600A200B3CC
:104486004006A202B3B3500990001EE4F0A3F080E8
:1044960024AE52AF537400D39F74019E400C90001B
:1044A6001EE552F0A3E553F0800B74FF90001EF852
:1044B600E4F0E8A3F09000C3E0D394024006A2081B
:1044C600B3B34002800DAE52AF5374021254768ECF
:1044D600528F539000ACE0B4010DAE52AF5374024C
:1044E6001254768E528F53AE52AF53745E12547678
:1044F600740A8E048F05FF1254588C528D53740221
:10450600BC000AD39D400675530275520090001CEC
:10451600E552F0A3E553F02290004DE090037B12A4
:1045260054A8E0F56775686490004DE0FE9000B70A
:10453600E0D39E4037E53875F00884FF7E008F5D36
:10454600E53875F00884ADF07C008D6075650875FA
:104556003303753496E55DC3941F50051238D98030
:1045660006900430E0F55D855D688035E53875F0C8
:104576000884FF7E008F5DE53875F00884ADF07C19
:10458600008D607565087533037534B6E55DC394B3
:104596001F50051238D98006900450E0F55D855D00
:1045A60068229000EDE0F562756511753304753487
:1045B60000AE25AF26E56275F00FA4FDACF0EDD395
:1045C6009FEC9E4021E5628E048F05FF125458ED44
:1045D60075F010A4FFAEF0E53875F01184FD7C008F
:1045E600ED2FF563800EE53875F01184FF7E00EF40
:1045F60024F0F56385635DE53875F01184AFF07ED0
:10460600008F601238D9855D64AE25AF269000ED27
:10461600E075F00FA4FDACF0EDD39FEC9E4028753D
:10462600330475341085635D1238D985645E855D03
:104636005FAE25AF26E5628E048F05FF1254918D7D
:1046460060856261123953855D67756864229000E2
:10465600EDE0F562756511753304753400AE25AF6E
:1046660026E56275F00FA4FDACF0EDD39FEC9E40FD
:1046760021E5628E048F05FF125458ED75F010A4E3
:10468600FFAEF0E53A75F01184FD7C00ED2FF56381
:10469600800EE53A75F01184FF7E00EF24F0F56395
:1046A60085635DE53A75F01184AFF07E008F601288
:1046B60038D9855D64AE25AF269000EDE075F00F24
:1046C600A4FDACF0EDD39FEC9E4028753304753401
:1046D6001085635D1238D985645E855D5FAE25AF52
:1046E60026E5628E048F05FF1254918D6085626106
:1046F600123953855D677568649000E8E0B4047903
:1047060090004DE0FE9000B7E0D39E4037E5387547
:10471600F00884FF7E008F5DE53875F00884ADF003
:104726007C008D60756508753303753496E55DC349
:10473600941F50051238D98006900430E0F55D8547
:104746005D688035E53875F00884FF7E008F5DE58D
:104756003875F00884ADF07C008D6075650875339A
:10476600037534B6E55DC3941F50051238D980062B
:10477600900450E0F55D855D6822900081E0B4010B
:104786003BE54075F00584FF7E008F5DE54075F0E2
:104796000584ADF07C008D6075650575330575344F
:1047A60018E55DC3941750051238D980069005AAFE
:1047B600E0F55DE568255DC39464F568900082E0E8
:1047C600B4013BE54175F00584FF7E008F5DE54150
:1047D60075F00584ADF07C008D6075650575330553
:1047E600753460E55DC3941750051238D98006907C
:1047F60005F2E0F55DE568255DC39464F568E56757
:104806002568F55A900089E0B402109007BFE025AC
:104816005AFE9000DDE0F4042EF55A9000E0E0D355
:1048260094014040E544C394E7501D74E7C39544A2
:10483600FE9007C1E08E00F5F0E884FF7E008F5DF4
:10484600E55A255DF55A801CE544C394E7FE9007BA
:10485600C1E08E00F5F0E884FF7E008F5DE55AC367
:10486600955DF55AA2084006E5672464F55AE55AAF
:10487600D394644009E55AC39464F55A8003755A83
:10488600009000B9E0C3955A50069000B9E0F55A79
:1048960022D2009000CFE0A825B800049526503B10
:1048A6009000CFE0A825B8000495265003755A0F4E
:1048B6009000CFE004A825B8000495265003755A49
:1048C6000A9000CFE02402A825B8000495265005DA
:1048D600755A05C2007409900050F07E017F009061
:1048E60000BFE01254769000CEE08E048F05FF12D2
:1048F6005458E538BC000CD39D4008C200740A9099
:104906000050F09000C0E0C39540500D9000D2E0FA
:10491600A825B80006952640028008C200740B90B0
:104926000050F0A2004003755A05900089E0B403D8
:1049360006A201B3B34002802B900075E0C3940534
:10494600A825B800049526500C9000AAE0F55A74E4
:104956000C900050F0900075E0A825B8000495264C
:104966005002C200855A4590007BE0255AFE900011
:104976004DE075F01E84FC7F00EE2CF55A22900067
:104986004DE075F00584FF7E008F5D90004DE0756B
:10499600F00584ADF07C008D607565057533037593
:1049A60034D69000CCE01475F00584FF7E00E55DFA
:1049B600BE00039F50051238D9800BE55D90045167
:1049C6001254A8E0F55DE55D9007C2F09007C2E0DD
:1049D600FE9000BBE0C39E50089000BBE09007C26B
:1049E600F022E54075F00584FF7E0090057B1254A9
:1049F6009DE0F56CE56CD394644010E56CC394645B
:104A060075F00F84FF7E008F6C8003756C0090003C
:104A16009EE0256CF56C229007B5E0FEA3E0FF74DE
:104A260004125468E538125476740F8E048F05FF0D
:104A36001254589007B3ECF0A3EDF0900091E0B457
:104A46000262E543C3944175F00584FF7E008F5DE5
:104A5600E54375F00584ADF07C008D6075650575E0
:104A66003306753414E55DC3941750051238D980A2
:104A7600069006A2E0F55D9007B3E0FEA3E0FF74A2
:104A86000A8E048F05FF125458E55D8C068D0712B9
:104A96005476740A8E048F05FF1254589007B3ECAF
:104AA600F0A3EDF09007B3E0FEA3E0FF9007B9E0B6
:104AB600FCA3E0FDEDD39FEC9E400F9007B9E0F814
:104AC600A3E09007B3C8F0A3C8F022900098E0B422
:104AD6000103852650900098E0B402129000CEE0C3
:104AE6008538F0A4FFAEF074081254688F50900019
:104AF60098E0B40303853A50900098E0B404038527
:104B06004050900098E0B40503854150900098E02D
:104B1600B40603854250900098E0B40703854350DD
:104B2600900098E0B40803854450900098E0B409DA
:104B360003853F50900098E0B40A03853E509000EC
:104B460098E0B40B03854550900098E0B40C0690AD
:104B5600001FE0F550900099E0FE90009AE0D39E89
:104B6600404B900098E0B4041890009AE0C395502A
:104B76005002D204900099E0D395504002C20480BE
:104B86002A900099E0C39550500990009AE0D39579
:104B96005050028002D204900099E0D395505009FB
:104BA60090009AE0C395505002C204802A90009962
:104BB600E0D39550400990009AE0C395504002809A
:104BC60002C204900099E0C39550400990009AE013
:104BD600D395504002D2042290009BE0B401038595
:104BE600265090009BE0B402129000CEE08538F08B
:104BF600A4FFAEF074081254688F5090009BE0B486
:104C06000303853A5090009BE0B40403854050901E
:104C1600009BE0B4050385415090009BE0B4060379
:104C260085425090009BE0B4070385435090009B5B
:104C3600E0B4080385445090009BE0B40903853F27
:104C46005090009BE0B40A03853E5090009BE0B470
:104C56000B0385455090009BE0B40C0690001FE0C6
:104C6600F55090009CE0FE90009DE0D39E40409061
:104C7600009CE0C39550500990009DE0D39550509C
:104C8600028002D20690009CE0D395505009900015
:104C96009DE0C395505002C20690009BE0B4010906
:104CA6009000DAE0D3953A50028002C206802A903C
:104CB600009CE0D39550400990009DE0C39550407C
:104CC600028002C20690009CE0C395504009900005
:104CD6009DE0D395504002D20622AE58AF5974F5E6
:104CE600D39F74019E400878581254D3024DFA752A
:104CF6005901755800AE25AF26E56CBE000DD39F51
:104D060040099000B0E0D3956D40028023756D0098
:104D1600E56CC39526F5509000B3E0D3956B40083B
:104D2600E56B2550F56B80069000B3E0F56B8002CD
:104D3600056D90008CE0D3953A401CE538C3953953
:104D46004015AE25AF26E56CBE00039F50099000C6
:104D5600B1E0D3956E4002806E9007C3E0A825B8F7
:104D66000004952650037570009007C3E0A825B887
:104D7600000BD395264006E5269007C3F0E5707034
:104D860041E526C3956CF550E550D394054003756F
:104D960050059000B2E0C3956B5007E550C3956B84
:104DA60040028009E56BC39550F56B80069000B212
:104DB600E0F56B9000B2E0D3956B40069000B2E050
:104DC600F56B756E008002056EE570701690008CAE
:104DD600E0C3953A500DE56C2405A825B800069564
:104DE600264002800F90009FE0F56B757001747885
:104DF6009007C3F022AE58AF5974E9D39F74039E4F
:104E0600400878581254D3024F99755901755800C5
:104E1600756B32A226402A756B1990009FE075F0DB
:104E260002A4FFAEF0E56DBE0006D39F4002D22677
:104E3600056D75700374789007C3F0756F00024FA7
:104E460088AE25AF26E56C6F4E7003024F88E56C81
:104E5600BE000DD39F40099000B0E0D3956D40028F
:104E6600800F756D00E570C394035003756B198050
:104E76000DE56CC39526F550E56D2550F56D900052
:104E86008CE0D3953A400E9007C3E0A825B80007FA
:104E9600D395264002800C056F90009FE0B56F0306
:104EA600757000E570B40306A208B3B34002800A29
:104EB600056FE56FB43C03757002E570B402299086
:104EC60007C3E0A825B8000ED395264009E526902D
:104ED60007C3F0756F0090008CE0C3953A500975D2
:104EE6006F0074789007C3F0E570705A90008CE0FC
:104EF600D3953A401CE538D395394015AE25AF26F3
:104F0600E56CBE00039F50099000B1E0D3956E405A
:104F1600028008756E00756B4B8028E526C3956C7C
:104F2600F550E550D39405400375500590008CE08C
:104F3600D3953A4008E56E2550F56E8006E56E2459
:104F460006F56E756F00E570701690008CE0C395DF
:104F56003A500DE56C2405A825B8000695264002B2
:104F66008003757001E570B40118756B19056F90B3
:104F7600009FE0B56F06757002756F007478900734
:104F8600C3F0E56B75F00AA4FFAEF09007BDEEF036
:044F9600A3EFF02273
:0954A8002582F5825002058322E1
:0F008C0025E050020583258250020583F582226C
:10543700EF2F500205832582F582E5833E2EF58303
:015447002242
:1054C300CFC39FFF50011E22C3EF9DFFEE9CFE2220
:0954B100E493F608740193F6225D
:0854D3000806B60002180622CB
:0D548400A3E004F07006120049E004F022DD
:0E003900A3E014F0B4FF06120049E014F02218
:0E546800048007C3CE13CECF13CFD5E0F622BB
:10535600BC000FBE0008ED8FF084FFADF022E4FE26
:10536600FF22BE000DEF60FE54F0606F20E70302DF
:10537600540CEAC0E0EBC0E078017A0075F001EE6B
:1053860020E710EF25E0FFEE33FE0AC5F023C5F057
:1053960030E7F0EA5407F9096A7A007B00600108F1
:1053A600C3EC9E40167004ED9F4010ED9FFDEC9EF1
:1053B600FCE5F0CA4ACA03F5F08005E5F003F5F00E
:1053C600C3EE13FEEF13FFD9D77908CACBCAD8D0DC
:1053D600EAFEEBFFD0E0FBD0E0FA22EC8FF084FC93
:1053E600ED54F045F0C48FF084FEEDC454F045F062
:1053F600C48FF084FDEEC4FE54F02DFFEE540F3C36
:10540600FEADF07C0022790078008FF0EC7E08205B
:10541600E70DC3CD33CD33C933C9C833C8DEF084F5
:1054260049F9E5F08FF0BE00E6FD7C00E9FFE8FEF5
:015436002253
:0E547600F88FF0A4FFE5F0CE88F0A42EFE2201
:10000300EF8DF0A4F9A8F0EF8CF0A428F8EE8DF0B2
:06001300A428FEE9FF2213
:10544800600D782B025452007830D8FED5E0F8224F
:10545800EEC0E07E00125356EFFDEEFCD0E0FE22D7
:0C549100EEC0E07E00125356D0E0FE2278
:03001B0002001EC2
:0300530002005652
:03009B00020071EF
:030000000254BAED
:0954BA0075817175D00002066BCA
:0B549D00E5822FF582E5833EF58322B7
:0A0049000582D5820215831582227C
:10001E00C0E0C0F0C083C082C0D075D0001205C64B
:0B002E00D0D0D082D083D0F0D0E032E0
:10005600C0E0C0F0C083C082C0D075D0001205C910
:10006600D0D0D082D083D0F0D0E032C0E0C0F0C093
:1000760083C082C0D075D000120633D0D0D082D0D3
:0600860083D0F0D0E0324F
:00000001FF
